******************************************************************************
             TMS320C2000 Linker PC v6.1.0                      
******************************************************************************
>> Linked Fri Nov 06 10:41:14 2020

OUTPUT FILE NAME:   <test_adc.out>
ENTRY POINT SYMBOL: "_c_int00"  address: 00339d1e


MEMORY CONFIGURATION

         name            origin    length      used     unused   attr    fill
----------------------  --------  ---------  --------  --------  ----  --------
PAGE 0:
  ZONE0                 00004000   00001000  00000000  00001000  RWIX
  RAML0                 00008000   00001000  000001c4  00000e3c  RWIX
  RAML1                 00009000   00001000  00000000  00001000  RWIX
  RAML2                 0000a000   00001000  00000000  00001000  RWIX
  RAML3                 0000b000   00001000  00000000  00001000  RWIX
  ZONE6                 00100000   00100000  00000000  00100000  RWIX
  ZONE7A                00200000   0000fc00  00000000  0000fc00  RWIX
  FLASHH                00300000   00008000  00000000  00008000  RWIX
  FLASHG                00308000   00008000  00000000  00008000  RWIX
  FLASHF                00310000   00008000  00000000  00008000  RWIX
  FLASHE                00318000   00008000  00000000  00008000  RWIX
  FLASHD                00320000   00008000  000001c4  00007e3c  RWIX
  FLASHC                00328000   00008000  00000000  00008000  RWIX
  FLASHA                00338000   00007f80  0000215e  00005e22  RWIX
  CSM_RSVD              0033ff80   00000076  00000000  00000076  RWIX
  BEGIN                 0033fff6   00000002  00000002  00000000  RWIX
  CSM_PWL               0033fff8   00000008  00000000  00000008  RWIX
  ADC_CAL               00380080   00000009  00000007  00000002  RWIX
  OTP                   00380400   00000400  00000000  00000400  RWIX
  IQTABLES              003fe000   00000b50  00000000  00000b50  RWIX
  IQTABLES2             003feb50   0000008c  00000000  0000008c  RWIX
  FPUTABLES             003febdc   000006a0  00000000  000006a0  RWIX
  ROM                   003ff27c   00000d44  00000000  00000d44  RWIX
  RESET                 003fffc0   00000002  00000000  00000002  RWIX
  VECTORS               003fffc2   0000003e  00000000  0000003e  RWIX

PAGE 1:
  BOOT_RSVD             00000000   00000050  00000050  00000000  RWIX
  RAMM0                 00000050   000003b0  000003af  00000001  RWIX
  RAMM1                 00000400   00000400  00000400  00000000  RWIX
  RAML4                 0000c000   00001000  00000af6  0000050a  RWIX
  RAML5                 0000d000   00001000  00000000  00001000  RWIX
  RAML6                 0000e000   00001000  00000000  00001000  RWIX
  RAML7                 0000f000   00001000  00000000  00001000  RWIX
  ZONE7B                0020fc00   00000400  00000000  00000400  RWIX
  FLASHB                00330000   00008000  00000000  00008000  RWIX


SECTION ALLOCATION MAP

 output                                  attributes/
section   page    origin      length       input sections
--------  ----  ----------  ----------   ----------------
.pinit     0    00338000    00000000     UNINITIALIZED

ramfuncs   0    00320000    000001c4     RUN ADDR = 00008000
                  00320000    00000120     adc.obj (ramfuncs)
                  00320120    00000051     F28335Port.obj (ramfuncs)
                  00320171    00000020     SystemTrap.obj (ramfuncs)
                  00320191    0000001b     DSP2833x_SysCtrl.obj (ramfuncs)
                  003201ac    00000014     DSP2833x_DMA.obj (ramfuncs)
                  003201c0    00000004     DSP2833x_usDelay.obj (ramfuncs)

.text      0    00338000    00001eda     
                  00338000    00000503     F28335Epwm.obj (.text)
                  00338503    000004ea     F28335Adc.obj (.text)
                  003389ed    000003f5     DSP2833x_DMA.obj (.text)
                  00338de2    00000316     DSP2833x_DefaultIsr.obj (.text:retain)
                  003390f8    000002bc     DSP2833x_EPwm.obj (.text)
                  003393b4    000001d4     rts2800_fpu32.lib : memory.obj (.text)
                  00339588    0000016c     DSP2833x_Mcbsp.obj (.text)
                  003396f4    00000134     DSP2833x_ECan.obj (.text)
                  00339828    000000f6     DSP2833x_Xintf.obj (.text)
                  0033991e    000000f3     DSP2833x_SysCtrl.obj (.text)
                  00339a11    00000080     DSP2833x_Adc.obj (.text)
                  00339a91    0000006e     DSP2833x_ECap.obj (.text)
                  00339aff    0000006c     F28335Port.obj (.text)
                  00339b6b    00000066     adc.obj (.text)
                  00339bd1    0000005f     SystemTrap.obj (.text)
                  00339c30    00000056     DSP2833x_EQep.obj (.text)
                  00339c86    00000051     DSP2833x_CpuTimers.obj (.text)
                  00339cd7    00000047     DSP2833x_Sci.obj (.text)
                  00339d1e    00000046     rts2800_fpu32.lib : boot.obj (.text)
                  00339d64    00000032     main.obj (.text)
                  00339d96    00000028     DSP2833x_PieCtrl.obj (.text)
                  00339dbe    00000026     DSP2833x_Spi.obj (.text)
                  00339de4    00000021     rts2800_fpu32.lib : memcpy_ff.obj (.text)
                  00339e05    00000020     DSP2833x_PieVect.obj (.text)
                  00339e25    0000001f     rts2800_fpu32.lib : new_.obj (.text)
                  00339e44    00000019                       : args_main.obj (.text)
                  00339e5d    00000019                       : exit.obj (.text)
                  00339e76    00000017     DSP2833x_Gpio.obj (.text)
                  00339e8d    00000017     DSP2833x_I2C.obj (.text)
                  00339ea4    00000015     DSP2833x_MemCopy.obj (.text)
                  00339eb9    00000009     rts2800_fpu32.lib : _lock.obj (.text)
                  00339ec2    00000008     DSP2833x_CodeStartBranch.obj (.text)
                  00339eca    00000007     DSP2833x_DisInt.obj (.text)
                  00339ed1    00000005     rts2800_fpu32.lib : delete.obj (.text)
                  00339ed6    00000003     DSP2833x_DBGIER.obj (.text)
                  00339ed9    00000001     rts2800_fpu32.lib : newhandler.obj (.text)

.cinit     0    00339eda    0000014c     
                  00339eda    000000a3     F28335Adc.obj (.cinit)
                  00339f7d    00000086     adc.obj (.cinit)
                  0033a003    0000000a     rts2800_fpu32.lib : _lock.obj (.cinit)
                  0033a00d    0000000a                       : exit.obj (.cinit)
                  0033a017    00000005                       : vars.obj (.cinit)
                  0033a01c    00000004     SystemTrap.obj (.cinit)
                  0033a020    00000004     rts2800_fpu32.lib : memory.obj (.cinit)
                  0033a024    00000002     --HOLE-- [fill = 0]

.econst    0    0033a026    00000138     
                  0033a026    00000100     DSP2833x_PieVect.obj (.econst)
                  0033a126    00000038     F28335Adc.obj (.econst)

codestart 
*          0    0033fff6    00000002     
                  0033fff6    00000002     DSP2833x_CodeStartBranch.obj (codestart)

.adc_cal   0    00380080    00000007     NOLOAD SECTION
                  00380080    00000007     DSP2833x_ADC_cal.obj (.adc_cal)

.reset     0    003fffc0    00000002     DSECT
                  003fffc0    00000002     rts2800_fpu32.lib : boot.obj (.reset)

vectors    0    003fffc2    00000000     DSECT

ECanaLAMRegsFile 
*          1    00000000    00000040     UNINITIALIZED
                  00000000    00000040     DSP2833x_GlobalVariableDefs.obj (ECanaLAMRegsFile)

AdcMirrorFile 
*          1    00000040    00000010     UNINITIALIZED
                  00000040    00000010     DSP2833x_GlobalVariableDefs.obj (AdcMirrorFile)

GpioCtrlRegsFile 
*          1    00000050    0000002e     UNINITIALIZED
                  00000050    0000002e     DSP2833x_GlobalVariableDefs.obj (GpioCtrlRegsFile)

PartIdRegsFile 
*          1    0000007e    00000001     UNINITIALIZED
                  0000007e    00000001     DSP2833x_GlobalVariableDefs.obj (PartIdRegsFile)

ECanaMboxesFile 
*          1    00000080    00000100     UNINITIALIZED
                  00000080    00000100     DSP2833x_GlobalVariableDefs.obj (ECanaMboxesFile)

ECanbMboxesFile 
*          1    00000180    00000100     UNINITIALIZED
                  00000180    00000100     DSP2833x_GlobalVariableDefs.obj (ECanbMboxesFile)

PieVectTableFile 
*          1    00000280    00000100     UNINITIALIZED
                  00000280    00000100     DSP2833x_GlobalVariableDefs.obj (PieVectTableFile)

ECanaMOTORegsFile 
*          1    00000380    00000040     UNINITIALIZED
                  00000380    00000040     DSP2833x_GlobalVariableDefs.obj (ECanaMOTORegsFile)

ECanaMOTSRegsFile 
*          1    000003c0    00000040     UNINITIALIZED
                  000003c0    00000040     DSP2833x_GlobalVariableDefs.obj (ECanaMOTSRegsFile)

.stack     1    00000400    00000300     UNINITIALIZED
                  00000400    00000300     --HOLE--

DmaRegsFile 
*          1    00000700    000000e0     UNINITIALIZED
                  00000700    000000e0     DSP2833x_GlobalVariableDefs.obj (DmaRegsFile)

ECap1RegsFile 
*          1    000007e0    00000020     UNINITIALIZED
                  000007e0    00000020     DSP2833x_GlobalVariableDefs.obj (ECap1RegsFile)

.ebss      1    0000c000    0000017e     UNINITIALIZED
                  0000c000    00000108     adc.obj (.ebss)
                  0000c108    00000018     DSP2833x_CpuTimers.obj (.ebss)
                  0000c120    0000000c     F28335Port.obj (.ebss)
                  0000c12c    00000008     rts2800_fpu32.lib : memory.obj (.ebss)
                  0000c134    00000004                       : _lock.obj (.ebss)
                  0000c138    00000004                       : exit.obj (.ebss)
                  0000c13c    00000002                       : vars.obj (.ebss)
                  0000c13e    00000001     SystemTrap.obj (.ebss)
                  0000c13f    00000001     --HOLE--
                  0000c140    0000003e     F28335Adc.obj (.ebss)

.sysmem    1    0000c17e    00000400     UNINITIALIZED
                  0000c17e    00000001     rts2800_fpu32.lib : memory.obj (.sysmem)
                  0000c17f    000003ff     --HOLE--

DevEmuRegsFile 
*          1    0000c580    000000d0     UNINITIALIZED
                  0000c580    000000d0     DSP2833x_GlobalVariableDefs.obj (DevEmuRegsFile)

McbspaRegsFile 
*          1    0000c650    00000025     UNINITIALIZED
                  0000c650    00000025     DSP2833x_GlobalVariableDefs.obj (McbspaRegsFile)

GpioIntRegsFile 
*          1    0000c676    0000000a     UNINITIALIZED
                  0000c676    0000000a     DSP2833x_GlobalVariableDefs.obj (GpioIntRegsFile)

ECanbLAMRegsFile 
*          1    0000c680    00000040     UNINITIALIZED
                  0000c680    00000040     DSP2833x_GlobalVariableDefs.obj (ECanbLAMRegsFile)

ECanbMOTORegsFile 
*          1    0000c6c0    00000040     UNINITIALIZED
                  0000c6c0    00000040     DSP2833x_GlobalVariableDefs.obj (ECanbMOTORegsFile)

ECanbMOTSRegsFile 
*          1    0000c700    00000040     UNINITIALIZED
                  0000c700    00000040     DSP2833x_GlobalVariableDefs.obj (ECanbMOTSRegsFile)

EQep1RegsFile 
*          1    0000c740    00000040     UNINITIALIZED
                  0000c740    00000040     DSP2833x_GlobalVariableDefs.obj (EQep1RegsFile)

EQep2RegsFile 
*          1    0000c780    00000040     UNINITIALIZED
                  0000c780    00000040     DSP2833x_GlobalVariableDefs.obj (EQep2RegsFile)

ECanaRegsFile 
*          1    0000c7c0    00000034     UNINITIALIZED
                  0000c7c0    00000034     DSP2833x_GlobalVariableDefs.obj (ECanaRegsFile)

CpuTimer0RegsFile 
*          1    0000c7f4    00000008     UNINITIALIZED
                  0000c7f4    00000008     DSP2833x_GlobalVariableDefs.obj (CpuTimer0RegsFile)

ECanbRegsFile 
*          1    0000c800    00000034     UNINITIALIZED
                  0000c800    00000034     DSP2833x_GlobalVariableDefs.obj (ECanbRegsFile)

CpuTimer1RegsFile 
*          1    0000c834    00000008     UNINITIALIZED
                  0000c834    00000008     DSP2833x_GlobalVariableDefs.obj (CpuTimer1RegsFile)

McbspbRegsFile 
*          1    0000c840    00000025     UNINITIALIZED
                  0000c840    00000025     DSP2833x_GlobalVariableDefs.obj (McbspbRegsFile)

PieCtrlRegsFile 
*          1    0000c865    0000001a     UNINITIALIZED
                  0000c865    0000001a     DSP2833x_GlobalVariableDefs.obj (PieCtrlRegsFile)

EPwm1RegsFile 
*          1    0000c880    00000022     UNINITIALIZED
                  0000c880    00000022     DSP2833x_GlobalVariableDefs.obj (EPwm1RegsFile)

AdcRegsFile 
*          1    0000c8a2    0000001e     UNINITIALIZED
                  0000c8a2    0000001e     DSP2833x_GlobalVariableDefs.obj (AdcRegsFile)

EPwm2RegsFile 
*          1    0000c8c0    00000022     UNINITIALIZED
                  0000c8c0    00000022     DSP2833x_GlobalVariableDefs.obj (EPwm2RegsFile)

XintfRegsFile 
*          1    0000c8e2    0000001e     UNINITIALIZED
                  0000c8e2    0000001e     DSP2833x_GlobalVariableDefs.obj (XintfRegsFile)

EPwm3RegsFile 
*          1    0000c900    00000022     UNINITIALIZED
                  0000c900    00000022     DSP2833x_GlobalVariableDefs.obj (EPwm3RegsFile)

CsmRegsFile 
*          1    0000c922    00000010     UNINITIALIZED
                  0000c922    00000010     DSP2833x_GlobalVariableDefs.obj (CsmRegsFile)

CpuTimer2RegsFile 
*          1    0000c932    00000008     UNINITIALIZED
                  0000c932    00000008     DSP2833x_GlobalVariableDefs.obj (CpuTimer2RegsFile)

EPwm4RegsFile 
*          1    0000c940    00000022     UNINITIALIZED
                  0000c940    00000022     DSP2833x_GlobalVariableDefs.obj (EPwm4RegsFile)

SciaRegsFile 
*          1    0000c962    00000010     UNINITIALIZED
                  0000c962    00000010     DSP2833x_GlobalVariableDefs.obj (SciaRegsFile)

CsmPwlFile 
*          1    0000c972    00000008     UNINITIALIZED
                  0000c972    00000008     DSP2833x_GlobalVariableDefs.obj (CsmPwlFile)

EPwm5RegsFile 
*          1    0000c980    00000022     UNINITIALIZED
                  0000c980    00000022     DSP2833x_GlobalVariableDefs.obj (EPwm5RegsFile)

ScibRegsFile 
*          1    0000c9a2    00000010     UNINITIALIZED
                  0000c9a2    00000010     DSP2833x_GlobalVariableDefs.obj (ScibRegsFile)

FlashRegsFile 
*          1    0000c9b2    00000008     UNINITIALIZED
                  0000c9b2    00000008     DSP2833x_GlobalVariableDefs.obj (FlashRegsFile)

EPwm6RegsFile 
*          1    0000c9c0    00000022     UNINITIALIZED
                  0000c9c0    00000022     DSP2833x_GlobalVariableDefs.obj (EPwm6RegsFile)

ScicRegsFile 
*          1    0000c9e2    00000010     UNINITIALIZED
                  0000c9e2    00000010     DSP2833x_GlobalVariableDefs.obj (ScicRegsFile)

I2caRegsFile 
*          1    0000ca00    00000022     UNINITIALIZED
                  0000ca00    00000022     DSP2833x_GlobalVariableDefs.obj (I2caRegsFile)

SpiaRegsFile 
*          1    0000ca22    00000010     UNINITIALIZED
                  0000ca22    00000010     DSP2833x_GlobalVariableDefs.obj (SpiaRegsFile)

ECap2RegsFile 
*          1    0000ca40    00000020     UNINITIALIZED
                  0000ca40    00000020     DSP2833x_GlobalVariableDefs.obj (ECap2RegsFile)

ECap3RegsFile 
*          1    0000ca60    00000020     UNINITIALIZED
                  0000ca60    00000020     DSP2833x_GlobalVariableDefs.obj (ECap3RegsFile)

ECap4RegsFile 
*          1    0000ca80    00000020     UNINITIALIZED
                  0000ca80    00000020     DSP2833x_GlobalVariableDefs.obj (ECap4RegsFile)

ECap5RegsFile 
*          1    0000caa0    00000020     UNINITIALIZED
                  0000caa0    00000020     DSP2833x_GlobalVariableDefs.obj (ECap5RegsFile)

ECap6RegsFile 
*          1    0000cac0    00000020     UNINITIALIZED
                  0000cac0    00000020     DSP2833x_GlobalVariableDefs.obj (ECap6RegsFile)

GpioDataRegsFile 
*          1    0000cae0    00000020     UNINITIALIZED
                  0000cae0    00000020     DSP2833x_GlobalVariableDefs.obj (GpioDataRegsFile)

SysCtrlRegsFile 
*          1    0000cb00    00000020     UNINITIALIZED
                  0000cb00    00000020     DSP2833x_GlobalVariableDefs.obj (SysCtrlRegsFile)

XIntruptRegsFile 
*          1    0000cb20    00000010     UNINITIALIZED
                  0000cb20    00000010     DSP2833x_GlobalVariableDefs.obj (XIntruptRegsFile)


GLOBAL SYMBOLS: SORTED ALPHABETICALLY BY Name 

address    name
--------   ----
00338000   .text
00339e5d   C$$EXIT
00338ec8   _ADCINT_ISR
0000c004   _ADC_Peak_Conv_Comp
0000c002   _ADC_Valley_Conv_Comp
00380080   _ADC_cal
00000040   _AdcMirror
0000c8a2   _AdcRegs
0000c162   _Amb_Temp_Prev
00339c9c   _ConfigCpuTimer
0000c024   _Control_Fault_Code
0000c118   _CpuTimer0
0000c7f4   _CpuTimer0Regs
0000c108   _CpuTimer1
0000c834   _CpuTimer1Regs
0000c110   _CpuTimer2
0000c932   _CpuTimer2Regs
0000c972   _CsmPwl
0000c922   _CsmRegs
003399e0   _CsmUnlock
00338df6   _DATALOG_ISR
00338fea   _DINTCH1_ISR
00338ff4   _DINTCH2_ISR
00338ffe   _DINTCH3_ISR
00339008   _DINTCH4_ISR
00339012   _DINTCH5_ISR
0033901c   _DINTCH6_ISR
003389f8   _DMACH1AddrConfig
000081ac   _DMACH1AddrConfigAndStart
00338a0a   _DMACH1BurstConfig
00338a3d   _DMACH1ModeConfig
00338a1a   _DMACH1TransferConfig
00338a2a   _DMACH1WrapConfig
00338a9f   _DMACH2AddrConfig
00338ab1   _DMACH2BurstConfig
00338ae4   _DMACH2ModeConfig
00338ac1   _DMACH2TransferConfig
00338ad1   _DMACH2WrapConfig
00338b46   _DMACH3AddrConfig
00338b58   _DMACH3BurstConfig
00338b8b   _DMACH3ModeConfig
00338b68   _DMACH3TransferConfig
00338b78   _DMACH3WrapConfig
00338bed   _DMACH4AddrConfig
00338bff   _DMACH4BurstConfig
00338c32   _DMACH4ModeConfig
00338c0f   _DMACH4TransferConfig
00338c1f   _DMACH4WrapConfig
00338c94   _DMACH5AddrConfig
00338ca6   _DMACH5BurstConfig
00338cd9   _DMACH5ModeConfig
00338cb6   _DMACH5TransferConfig
00338cc6   _DMACH5WrapConfig
00338d3b   _DMACH6AddrConfig
00338d4d   _DMACH6BurstConfig
00338d80   _DMACH6ModeConfig
00338d5d   _DMACH6TransferConfig
00338d6d   _DMACH6WrapConfig
003389ed   _DMAInitialize
00339eca   _DSP28x_DisableInt
00339ece   _DSP28x_RestoreInt
000081c0   _DSP28x_usDelay
0000c126   _DSPInRegister
0000c120   _DSPOutRegister
0000c040   _Data_plot2
0000c580   _DevEmuRegs
00339931   _DisableDog
00339b50   _DisableUnusedPWMs
00339bff   _DisableWatchdog__Fv
00000700   _DmaRegs
00339076   _ECAN0INTA_ISR
0033908a   _ECAN0INTB_ISR
00339080   _ECAN1INTA_ISR
00339094   _ECAN1INTB_ISR
00338f5e   _ECAP1_INT_ISR
00338f68   _ECAP2_INT_ISR
00338f72   _ECAP3_INT_ISR
00338f7c   _ECAP4_INT_ISR
00338f86   _ECAP5_INT_ISR
00338f90   _ECAP6_INT_ISR
00000000   _ECanaLAMRegs
00000380   _ECanaMOTORegs
000003c0   _ECanaMOTSRegs
00000080   _ECanaMboxes
0000c7c0   _ECanaRegs
0000c680   _ECanbLAMRegs
0000c6c0   _ECanbMOTORegs
0000c700   _ECanbMOTSRegs
00000180   _ECanbMboxes
0000c800   _ECanbRegs
000007e0   _ECap1Regs
0000ca40   _ECap2Regs
0000ca60   _ECap3Regs
0000ca80   _ECap4Regs
0000caa0   _ECap5Regs
0000cac0   _ECap6Regs
00338e0a   _EMUINT_ISR
00338f22   _EPWM1_INT_ISR
00338ee6   _EPWM1_TZINT_ISR
00338f2c   _EPWM2_INT_ISR
00338ef0   _EPWM2_TZINT_ISR
00338f36   _EPWM3_INT_ISR
00338efa   _EPWM3_TZINT_ISR
00338f40   _EPWM4_INT_ISR
00338f04   _EPWM4_TZINT_ISR
00338f4a   _EPWM5_INT_ISR
00338f0e   _EPWM5_TZINT_ISR
00338f54   _EPWM6_INT_ISR
00338f18   _EPWM6_TZINT_ISR
00338373   _EPWM_GetEventTriggerInterruptStatus__F10pwm_base_t27epwm_event_trigger_select_t
00338034   _EPWM_SetCounterCompareValue__F10pwm_base_t29epwm_counter_compare_module_tUs
0033846e   _EPWM_SetDeadBandDelayCount__F10pwm_base_t26epwm_deadband_delay_mode_tUs
003380c9   _EPWM_SetEventTriggerInterruptEnable__F10pwm_base_t27epwm_event_trigger_enable_tb
00338242   _EPWM_SetEventTriggerSel__F10pwm_base_t27epwm_event_trigger_select_t25epwm_event_triggers_sel_t
00338000   _EPWM_SetTimeBaseCounter__F10pwm_base_tUs
0000c880   _EPwm1Regs
0000c8c0   _EPwm2Regs
0000c900   _EPwm3Regs
0000c940   _EPwm4Regs
0000c980   _EPwm5Regs
0000c9c0   _EPwm6Regs
00338f9a   _EQEP1_INT_ISR
00338fa4   _EQEP2_INT_ISR
0000c740   _EQep1Regs
0000c780   _EQep2Regs
00339db5   _EnableInterrupts
00008189   _ExternalInt2_isr
00339be6   _FastShutdown__Fv
0000c9b2   _FlashRegs
0000c02a   _GD_Pwr_Inv_A
0000c026   _GD_Pwr_Rec
0000c01c   _GPIO_test_flag
003383a8   _GetPWM1_Evnt_Trig_Status__F27epwm_event_trigger_select_t
003383c9   _GetPWM2_Evnt_Trig_Status__F27epwm_event_trigger_select_t
003383ea   _GetPWM3_Evnt_Trig_Status__F27epwm_event_trigger_select_t
0033840b   _GetPWM4_Evnt_Trig_Status__F27epwm_event_trigger_select_t
0033842c   _GetPWM5_Evnt_Trig_Status__F27epwm_event_trigger_select_t
0033844d   _GetPWM6_Evnt_Trig_Status__F27epwm_event_trigger_select_t
00338817   _Get_ADC_Channel_A0__F16adc_channel_a0_t
0033882d   _Get_ADC_Channel_A1__F16adc_channel_a1_t
00338843   _Get_ADC_Channel_A2__F16adc_channel_a2_t
00338859   _Get_ADC_Channel_A3__F16adc_channel_a3_t
0033886f   _Get_ADC_Channel_A4__F16adc_channel_a4_t
00338885   _Get_ADC_Channel_A5__F16adc_channel_a5_t
0033889b   _Get_ADC_Channel_A6__F16adc_channel_a6_t
003388bf   _Get_ADC_Channel_A7__F16adc_channel_a7_t
00338902   _Get_ADC_Channel_B0__F16adc_channel_b0_t
00338918   _Get_ADC_Channel_B1__F16adc_channel_b1_t
0033892e   _Get_ADC_Channel_B2__F16adc_channel_b2_t
00338944   _Get_ADC_Channel_B3__F16adc_channel_b3_t
0033895a   _Get_ADC_Channel_B4__F16adc_channel_b4_t
00338970   _Get_ADC_Channel_B5__F16adc_channel_b5_t
00338986   _Get_ADC_Channel_B6__F16adc_channel_b6_t
003389aa   _Get_ADC_Channel_B7__F16adc_channel_b7_t
0033871b   _Get_Amb_Temp__Fv
003387f3   _Get_IFB_GD_Inv_A__Fv
003387cf   _Get_IFB_GD_Rec__Fv
00338787   _Get_IFB_P12__Fv
0033873f   _Get_IFB_P15__Fv
003387ab   _Get_IFB_P24__Fv
00338763   _Get_IFB_P5__Fv
003385fb   _Get_Inv_Iac_A__Fv
003386f7   _Get_Inv_Temp_A__Fv
0033861f   _Get_Inv_Vac_A__Fv
003385b3   _Get_PLL_A__Fv
003385d7   _Get_Rec_Iac__Fv
003386d3   _Get_Rec_Temp__Fv
00338643   _Get_Rec_Vac__Fv
0033868b   _Get_Tap_P1_Iac__Fv
003386af   _Get_Tap_P2_Iac__Fv
00338667   _Get_Vdc__Fv
00000050   _GpioCtrlRegs
0000cae0   _GpioDataRegs
0000c676   _GpioIntRegs
00339026   _I2CINT1A_ISR
00339030   _I2CINT2A_ISR
0000ca00   _I2caRegs
0000c140   _IFB_Fltr_Reset
0000c158   _IFB_Fltr_Reset_Cond
0000c16a   _IFB_GD_Inv_A_Prev
0000c16e   _IFB_GD_Rec_Prev
0000c166   _IFB_P12_Prev
0000c16c   _IFB_P15_Prev
0000c168   _IFB_P24_Prev
0000c178   _IFB_P5_Prev
00338e1e   _ILLEGAL_ISR
00338de2   _INT13_ISR
00338dec   _INT14_ISR
0000c016   _I_Inv_A
0000c012   _I_Rec
0000c01a   _I_Tap_P1
0000c018   _I_Tap_P2
00008182   _Illegal_isr
00339a11   _InitAdc
00339c86   _InitCpuTimers
00339b09   _InitDSP_IORegs
003396f4   _InitECan
003397fd   _InitECanGpio
003396fb   _InitECana
00339802   _InitECanaGpio
0033977c   _InitECanb
00339818   _InitECanbGpio
00339a91   _InitECap
00339aa5   _InitECap1Gpio
00339ab3   _InitECap2Gpio
00339ac2   _InitECap3Gpio
00339ad0   _InitECap4Gpio
00339ade   _InitECap5Gpio
00339aec   _InitECap6Gpio
00339aa2   _InitECapGpio
00339c0b   _InitEPLDWatchdogEcho
003390f8   _InitEPwm
00339106   _InitEPwm1Gpio
00339118   _InitEPwm2Gpio
0033912a   _InitEPwm3Gpio
0033913e   _InitEPwm4Gpio
00339152   _InitEPwm5Gpio
00339164   _InitEPwm6Gpio
003390fd   _InitEPwmGpio
00339176   _InitEPwmTimer
00339c30   _InitEQep
00339c36   _InitEQep1Gpio
00339c60   _InitEQep2Gpio
00339c31   _InitEQepGpio
00008191   _InitFlash
00339e76   _InitGpio
00339e8d   _InitI2C
00339e8e   _InitI2CGpio
00339588   _InitMcbsp
00339661   _InitMcbspGpio
0033958d   _InitMcbspa
003395ec   _InitMcbspa12bit
003395f7   _InitMcbspa16bit
00339602   _InitMcbspa20bit
0033960d   _InitMcbspa24bit
00339618   _InitMcbspa32bit
003395e5   _InitMcbspa8bit
00339666   _InitMcbspaGpio
003395b9   _InitMcbspb
0033962a   _InitMcbspb12bit
00339635   _InitMcbspb16bit
00339640   _InitMcbspb20bit
0033964b   _InitMcbspb24bit
00339656   _InitMcbspb32bit
00339623   _InitMcbspb8bit
003396a0   _InitMcbspbGpio
00339985   _InitPeripheralClocks
00339d96   _InitPieCtrl
00339e05   _InitPieVectTable
00339939   _InitPll
00339a27   _InitProjectAdc
00339cd7   _InitSci
00339cd8   _InitSciGpio
00339cdf   _InitSciaGpio
00339cf4   _InitScibGpio
00339d08   _InitScicGpio
00339dbe   _InitSpi
00339dbf   _InitSpiGpio
00339dc2   _InitSpiaGpio
0033991e   _InitSysCtrl
00339bf1   _InitWatchdog
00339828   _InitXintf
003398c4   _InitXintf16Gpio
0033987d   _InitXintf32Gpio
0000c14a   _Inv_Iac_Prev
0000c154   _Inv_Temp_A_Prev
0000c17c   _Inv_Vac_Prev
00339b42   _InverterPWMOff
00339b2d   _InverterPWMOn
00008171   _KickWatchdog__Fv
003390da   _LUF_ISR
003390d0   _LVF_ISR
00338fd6   _MRINTA_ISR
00338fc2   _MRINTB_ISR
00338fe0   _MXINTA_ISR
00338fcc   _MXINTB_ISR
0000c650   _McbspaRegs
0000c840   _McbspbRegs
00339ea4   _MemCopy
00338e14   _NMI_ISR
003390e4   _PIE_RESERVED
0000c142   _PLLA_Fltr_Reset
0000c150   _PLLA_Fltr_Reset_Cond
0000c148   _PLL_CL7_Previous
0000c00a   _PS_12V
0000c008   _PS_1_5V
0000c02c   _PS_24V
0000c02e   _PS_5V
0000007e   _PartIdRegs
0000c001   _Peak_50ms_Even_Flag
0000c020   _Peak_Counter_50ms
0000c00e   _Phase_Locked_Loop_A
0000c865   _PieCtrlRegs
00000280   _PieVectTable
0033a026   _PieVectTableInit
00338e00   _RTOSINT_ISR
003201c4   _RamfuncsLoadEnd
00320000   _RamfuncsLoadStart
00008000   _RamfuncsRunStart
00008156   _ReadDSPInputs
0000c145   _Rec_Iac_Fltr_Reset
0000c14e   _Rec_Iac_Fltr_Reset_Cond
0000c14c   _Rec_Iac_Prev
0000c156   _Rec_Temp_Prev
0000c176   _Rec_Vac_Prev
0033904e   _SCIRXINTA_ISR
00339062   _SCIRXINTB_ISR
0033903a   _SCIRXINTC_ISR
00339058   _SCITXINTA_ISR
0033906c   _SCITXINTB_ISR
00339044   _SCITXINTC_ISR
00338ea0   _SEQ1INT_ISR
00338eaa   _SEQ2INT_ISR
00338fae   _SPIRXINTA_ISR
00338fb8   _SPITXINTA_ISR
0000c962   _SciaRegs
0000c9a2   _ScibRegs
0000c9e2   _ScicRegs
00339927   _ServiceDog
00339ed6   _SetDBGIER
00339b5c   _SetIOGood
00338069   _SetPWM1_Cmp_Val__F29epwm_counter_compare_module_tUs
003384a3   _SetPWM1_DB_Delay_Count__F26epwm_deadband_delay_mode_tUs
003380fe   _SetPWM1_Evnt_Trig_Int_Enable__F27epwm_event_trigger_enable_tb
00338277   _SetPWM1_Evnt_Trig_Select__F27epwm_event_trigger_select_t25epwm_event_triggers_sel_t
00338079   _SetPWM2_Cmp_Val__F29epwm_counter_compare_module_tUs
003384b3   _SetPWM2_DB_Delay_Count__F26epwm_deadband_delay_mode_tUs
00338134   _SetPWM2_Evnt_Trig_Int_Enable__F27epwm_event_trigger_enable_tb
003382a1   _SetPWM2_Evnt_Trig_Select__F27epwm_event_trigger_select_t25epwm_event_triggers_sel_t
00338089   _SetPWM3_Cmp_Val__F29epwm_counter_compare_module_tUs
003384c3   _SetPWM3_DB_Delay_Count__F26epwm_deadband_delay_mode_tUs
0033816a   _SetPWM3_Evnt_Trig_Int_Enable__F27epwm_event_trigger_enable_tb
003382cb   _SetPWM3_Evnt_Trig_Select__F27epwm_event_trigger_select_t25epwm_event_triggers_sel_t
00338099   _SetPWM4_Cmp_Val__F29epwm_counter_compare_module_tUs
003384d3   _SetPWM4_DB_Delay_Count__F26epwm_deadband_delay_mode_tUs
003381a0   _SetPWM4_Evnt_Trig_Int_Enable__F27epwm_event_trigger_enable_tb
003382f5   _SetPWM4_Evnt_Trig_Select__F27epwm_event_trigger_select_t25epwm_event_triggers_sel_t
003380a9   _SetPWM5_Cmp_Val__F29epwm_counter_compare_module_tUs
003384e3   _SetPWM5_DB_Delay_Count__F26epwm_deadband_delay_mode_tUs
003381d6   _SetPWM5_Evnt_Trig_Int_Enable__F27epwm_event_trigger_enable_tb
0033831f   _SetPWM5_Evnt_Trig_Select__F27epwm_event_trigger_select_t25epwm_event_triggers_sel_t
003380b9   _SetPWM6_Cmp_Val__F29epwm_counter_compare_module_tUs
003384f3   _SetPWM6_DB_Delay_Count__F26epwm_deadband_delay_mode_tUs
0033820c   _SetPWM6_Evnt_Trig_Int_Enable__F27epwm_event_trigger_enable_tb
00338349   _SetPWM6_Evnt_Trig_Select__F27epwm_event_trigger_select_t25epwm_event_triggers_sel_t
0000ca22   _SpiaRegs
00338a97   _StartDMACH1
00338b3e   _StartDMACH2
00338be5   _StartDMACH3
00338c8c   _StartDMACH4
00338d33   _StartDMACH5
00338dda   _StartDMACH6
00339afa   _StarteCAPTimers
003393ac   _StartePWMTimers
0000cb00   _SysCtrlRegs
00338ed2   _TINT0_ISR
0000c146   _TapIac_Fltr_Reset
0000c15a   _TapIac_Fltr_Reset_Cond
0000c170   _Tap_P1_Iac_Prev
0000c17a   _Tap_P2_Iac_Prev
0000c006   _Temp_Amb
0000c141   _Temp_Fltr_Reset
0000c152   _Temp_Fltr_Reset_Cond
0000c028   _Temp_Inv_A
0000c010   _Temp_Rec
00338e82   _USER10_ISR
00338e8c   _USER11_ISR
00338e96   _USER12_ISR
00338e28   _USER1_ISR
00338e32   _USER2_ISR
00338e3c   _USER3_ISR
00338e46   _USER4_ISR
00338e50   _USER5_ISR
00338e5a   _USER6_ISR
00338e64   _USER7_ISR
00338e6e   _USER8_ISR
00338e78   _USER9_ISR
00008000   _Update_Peripheral_Inputs__Fv
00008005   _Update_Peripheral_Outputs__Fv
0000c00c   _V_DC
0000c014   _V_Inv_A
0000c030   _V_Rec
0000c144   _Vac_Fltr_Reset
0000c15e   _Vac_Fltr_Reset_Cond
0000c005   _Valley_50ms_Even_Flag
0000c022   _Valley_Counter_50ms
0000c143   _Vdc_Fltr_Reset
0000c164   _Vdc_Fltr_Reset_Cond
0000c172   _Vdc_Prev
00338edc   _WAKEINT_ISR
00339bd1   _WatchdogReset__Fv
0000817b   _Watchdog_Overflow_isr
00008120   _WriteDSPOutputs_ISR
00338eb4   _XINT1_ISR
00338ebe   _XINT2_ISR
0033909e   _XINT3_ISR
003390a8   _XINT4_ISR
003390b2   _XINT5_ISR
003390bc   _XINT6_ISR
003390c6   _XINT7_ISR
0000cb20   _XIntruptRegs
0000c8e2   _XintfRegs
00000700   __STACK_END
00000300   __STACK_SIZE
00000400   __SYSMEM_SIZE
00000001   __TI_args_main
ffffffff   ___binit__
ffffffff   ___c_args__
00339eda   ___cinit__
00339ed9   ___default_new_handler__Fv
00339ed1   ___dl__FPv
00339eda   ___etext__
00339de4   ___memcpy_ff
00339e25   ___nw__FUl
ffffffff   ___pinit__
00338000   ___text__
00339e44   __args_main
0000c138   __cleanup_ptr
0000c13a   __dtors_ptr
0000c136   __lock
0000c13c   __new_handler
00339ec1   __nop
00339ebd   __register_lock
00339eb9   __register_unlock
00000400   __stack
0000c17e   __sys_memory
0000c134   __unlock
00339e5d   _abort
0000804a   _adc_isr
00339d1e   _c_int00
0033956e   _calloc
0033956c   _chkheap
003396de   _clkg_delay_loop
00008006   _control_isr
0000c000   _control_isr_val
003396c8   _delay_loop
00339e5f   _exit
003393b4   _free
0033954e   _free_memory
0000c160   _gAmplitude
0000c15c   _gSineDivisions
0000c003   _g_stopWatchdog
0000c174   _gsine_count
0000c032   _i
0000c01e   _initialization_flag
00339d64   _main
0033941f   _malloc
0033952c   _max_free
003393f9   _minit
00339475   _realloc
003390ee   _rsvd_ISR
0000c13e   _xi2Counter
ffffffff   binit
00339eda   cinit
0033fff6   code_start
00339eda   etext
ffffffff   pinit


GLOBAL SYMBOLS: SORTED BY Symbol Address 

address    name
--------   ----
00000000   _ECanaLAMRegs
00000001   __TI_args_main
00000040   _AdcMirror
00000050   _GpioCtrlRegs
0000007e   _PartIdRegs
00000080   _ECanaMboxes
00000180   _ECanbMboxes
00000280   _PieVectTable
00000300   __STACK_SIZE
00000380   _ECanaMOTORegs
000003c0   _ECanaMOTSRegs
00000400   __SYSMEM_SIZE
00000400   __stack
00000700   _DmaRegs
00000700   __STACK_END
000007e0   _ECap1Regs
00008000   _RamfuncsRunStart
00008000   _Update_Peripheral_Inputs__Fv
00008005   _Update_Peripheral_Outputs__Fv
00008006   _control_isr
0000804a   _adc_isr
00008120   _WriteDSPOutputs_ISR
00008156   _ReadDSPInputs
00008171   _KickWatchdog__Fv
0000817b   _Watchdog_Overflow_isr
00008182   _Illegal_isr
00008189   _ExternalInt2_isr
00008191   _InitFlash
000081ac   _DMACH1AddrConfigAndStart
000081c0   _DSP28x_usDelay
0000c000   _control_isr_val
0000c001   _Peak_50ms_Even_Flag
0000c002   _ADC_Valley_Conv_Comp
0000c003   _g_stopWatchdog
0000c004   _ADC_Peak_Conv_Comp
0000c005   _Valley_50ms_Even_Flag
0000c006   _Temp_Amb
0000c008   _PS_1_5V
0000c00a   _PS_12V
0000c00c   _V_DC
0000c00e   _Phase_Locked_Loop_A
0000c010   _Temp_Rec
0000c012   _I_Rec
0000c014   _V_Inv_A
0000c016   _I_Inv_A
0000c018   _I_Tap_P2
0000c01a   _I_Tap_P1
0000c01c   _GPIO_test_flag
0000c01e   _initialization_flag
0000c020   _Peak_Counter_50ms
0000c022   _Valley_Counter_50ms
0000c024   _Control_Fault_Code
0000c026   _GD_Pwr_Rec
0000c028   _Temp_Inv_A
0000c02a   _GD_Pwr_Inv_A
0000c02c   _PS_24V
0000c02e   _PS_5V
0000c030   _V_Rec
0000c032   _i
0000c040   _Data_plot2
0000c108   _CpuTimer1
0000c110   _CpuTimer2
0000c118   _CpuTimer0
0000c120   _DSPOutRegister
0000c126   _DSPInRegister
0000c134   __unlock
0000c136   __lock
0000c138   __cleanup_ptr
0000c13a   __dtors_ptr
0000c13c   __new_handler
0000c13e   _xi2Counter
0000c140   _IFB_Fltr_Reset
0000c141   _Temp_Fltr_Reset
0000c142   _PLLA_Fltr_Reset
0000c143   _Vdc_Fltr_Reset
0000c144   _Vac_Fltr_Reset
0000c145   _Rec_Iac_Fltr_Reset
0000c146   _TapIac_Fltr_Reset
0000c148   _PLL_CL7_Previous
0000c14a   _Inv_Iac_Prev
0000c14c   _Rec_Iac_Prev
0000c14e   _Rec_Iac_Fltr_Reset_Cond
0000c150   _PLLA_Fltr_Reset_Cond
0000c152   _Temp_Fltr_Reset_Cond
0000c154   _Inv_Temp_A_Prev
0000c156   _Rec_Temp_Prev
0000c158   _IFB_Fltr_Reset_Cond
0000c15a   _TapIac_Fltr_Reset_Cond
0000c15c   _gSineDivisions
0000c15e   _Vac_Fltr_Reset_Cond
0000c160   _gAmplitude
0000c162   _Amb_Temp_Prev
0000c164   _Vdc_Fltr_Reset_Cond
0000c166   _IFB_P12_Prev
0000c168   _IFB_P24_Prev
0000c16a   _IFB_GD_Inv_A_Prev
0000c16c   _IFB_P15_Prev
0000c16e   _IFB_GD_Rec_Prev
0000c170   _Tap_P1_Iac_Prev
0000c172   _Vdc_Prev
0000c174   _gsine_count
0000c176   _Rec_Vac_Prev
0000c178   _IFB_P5_Prev
0000c17a   _Tap_P2_Iac_Prev
0000c17c   _Inv_Vac_Prev
0000c17e   __sys_memory
0000c580   _DevEmuRegs
0000c650   _McbspaRegs
0000c676   _GpioIntRegs
0000c680   _ECanbLAMRegs
0000c6c0   _ECanbMOTORegs
0000c700   _ECanbMOTSRegs
0000c740   _EQep1Regs
0000c780   _EQep2Regs
0000c7c0   _ECanaRegs
0000c7f4   _CpuTimer0Regs
0000c800   _ECanbRegs
0000c834   _CpuTimer1Regs
0000c840   _McbspbRegs
0000c865   _PieCtrlRegs
0000c880   _EPwm1Regs
0000c8a2   _AdcRegs
0000c8c0   _EPwm2Regs
0000c8e2   _XintfRegs
0000c900   _EPwm3Regs
0000c922   _CsmRegs
0000c932   _CpuTimer2Regs
0000c940   _EPwm4Regs
0000c962   _SciaRegs
0000c972   _CsmPwl
0000c980   _EPwm5Regs
0000c9a2   _ScibRegs
0000c9b2   _FlashRegs
0000c9c0   _EPwm6Regs
0000c9e2   _ScicRegs
0000ca00   _I2caRegs
0000ca22   _SpiaRegs
0000ca40   _ECap2Regs
0000ca60   _ECap3Regs
0000ca80   _ECap4Regs
0000caa0   _ECap5Regs
0000cac0   _ECap6Regs
0000cae0   _GpioDataRegs
0000cb00   _SysCtrlRegs
0000cb20   _XIntruptRegs
00320000   _RamfuncsLoadStart
003201c4   _RamfuncsLoadEnd
00338000   .text
00338000   _EPWM_SetTimeBaseCounter__F10pwm_base_tUs
00338000   ___text__
00338034   _EPWM_SetCounterCompareValue__F10pwm_base_t29epwm_counter_compare_module_tUs
00338069   _SetPWM1_Cmp_Val__F29epwm_counter_compare_module_tUs
00338079   _SetPWM2_Cmp_Val__F29epwm_counter_compare_module_tUs
00338089   _SetPWM3_Cmp_Val__F29epwm_counter_compare_module_tUs
00338099   _SetPWM4_Cmp_Val__F29epwm_counter_compare_module_tUs
003380a9   _SetPWM5_Cmp_Val__F29epwm_counter_compare_module_tUs
003380b9   _SetPWM6_Cmp_Val__F29epwm_counter_compare_module_tUs
003380c9   _EPWM_SetEventTriggerInterruptEnable__F10pwm_base_t27epwm_event_trigger_enable_tb
003380fe   _SetPWM1_Evnt_Trig_Int_Enable__F27epwm_event_trigger_enable_tb
00338134   _SetPWM2_Evnt_Trig_Int_Enable__F27epwm_event_trigger_enable_tb
0033816a   _SetPWM3_Evnt_Trig_Int_Enable__F27epwm_event_trigger_enable_tb
003381a0   _SetPWM4_Evnt_Trig_Int_Enable__F27epwm_event_trigger_enable_tb
003381d6   _SetPWM5_Evnt_Trig_Int_Enable__F27epwm_event_trigger_enable_tb
0033820c   _SetPWM6_Evnt_Trig_Int_Enable__F27epwm_event_trigger_enable_tb
00338242   _EPWM_SetEventTriggerSel__F10pwm_base_t27epwm_event_trigger_select_t25epwm_event_triggers_sel_t
00338277   _SetPWM1_Evnt_Trig_Select__F27epwm_event_trigger_select_t25epwm_event_triggers_sel_t
003382a1   _SetPWM2_Evnt_Trig_Select__F27epwm_event_trigger_select_t25epwm_event_triggers_sel_t
003382cb   _SetPWM3_Evnt_Trig_Select__F27epwm_event_trigger_select_t25epwm_event_triggers_sel_t
003382f5   _SetPWM4_Evnt_Trig_Select__F27epwm_event_trigger_select_t25epwm_event_triggers_sel_t
0033831f   _SetPWM5_Evnt_Trig_Select__F27epwm_event_trigger_select_t25epwm_event_triggers_sel_t
00338349   _SetPWM6_Evnt_Trig_Select__F27epwm_event_trigger_select_t25epwm_event_triggers_sel_t
00338373   _EPWM_GetEventTriggerInterruptStatus__F10pwm_base_t27epwm_event_trigger_select_t
003383a8   _GetPWM1_Evnt_Trig_Status__F27epwm_event_trigger_select_t
003383c9   _GetPWM2_Evnt_Trig_Status__F27epwm_event_trigger_select_t
003383ea   _GetPWM3_Evnt_Trig_Status__F27epwm_event_trigger_select_t
0033840b   _GetPWM4_Evnt_Trig_Status__F27epwm_event_trigger_select_t
0033842c   _GetPWM5_Evnt_Trig_Status__F27epwm_event_trigger_select_t
0033844d   _GetPWM6_Evnt_Trig_Status__F27epwm_event_trigger_select_t
0033846e   _EPWM_SetDeadBandDelayCount__F10pwm_base_t26epwm_deadband_delay_mode_tUs
003384a3   _SetPWM1_DB_Delay_Count__F26epwm_deadband_delay_mode_tUs
003384b3   _SetPWM2_DB_Delay_Count__F26epwm_deadband_delay_mode_tUs
003384c3   _SetPWM3_DB_Delay_Count__F26epwm_deadband_delay_mode_tUs
003384d3   _SetPWM4_DB_Delay_Count__F26epwm_deadband_delay_mode_tUs
003384e3   _SetPWM5_DB_Delay_Count__F26epwm_deadband_delay_mode_tUs
003384f3   _SetPWM6_DB_Delay_Count__F26epwm_deadband_delay_mode_tUs
003385b3   _Get_PLL_A__Fv
003385d7   _Get_Rec_Iac__Fv
003385fb   _Get_Inv_Iac_A__Fv
0033861f   _Get_Inv_Vac_A__Fv
00338643   _Get_Rec_Vac__Fv
00338667   _Get_Vdc__Fv
0033868b   _Get_Tap_P1_Iac__Fv
003386af   _Get_Tap_P2_Iac__Fv
003386d3   _Get_Rec_Temp__Fv
003386f7   _Get_Inv_Temp_A__Fv
0033871b   _Get_Amb_Temp__Fv
0033873f   _Get_IFB_P15__Fv
00338763   _Get_IFB_P5__Fv
00338787   _Get_IFB_P12__Fv
003387ab   _Get_IFB_P24__Fv
003387cf   _Get_IFB_GD_Rec__Fv
003387f3   _Get_IFB_GD_Inv_A__Fv
00338817   _Get_ADC_Channel_A0__F16adc_channel_a0_t
0033882d   _Get_ADC_Channel_A1__F16adc_channel_a1_t
00338843   _Get_ADC_Channel_A2__F16adc_channel_a2_t
00338859   _Get_ADC_Channel_A3__F16adc_channel_a3_t
0033886f   _Get_ADC_Channel_A4__F16adc_channel_a4_t
00338885   _Get_ADC_Channel_A5__F16adc_channel_a5_t
0033889b   _Get_ADC_Channel_A6__F16adc_channel_a6_t
003388bf   _Get_ADC_Channel_A7__F16adc_channel_a7_t
00338902   _Get_ADC_Channel_B0__F16adc_channel_b0_t
00338918   _Get_ADC_Channel_B1__F16adc_channel_b1_t
0033892e   _Get_ADC_Channel_B2__F16adc_channel_b2_t
00338944   _Get_ADC_Channel_B3__F16adc_channel_b3_t
0033895a   _Get_ADC_Channel_B4__F16adc_channel_b4_t
00338970   _Get_ADC_Channel_B5__F16adc_channel_b5_t
00338986   _Get_ADC_Channel_B6__F16adc_channel_b6_t
003389aa   _Get_ADC_Channel_B7__F16adc_channel_b7_t
003389ed   _DMAInitialize
003389f8   _DMACH1AddrConfig
00338a0a   _DMACH1BurstConfig
00338a1a   _DMACH1TransferConfig
00338a2a   _DMACH1WrapConfig
00338a3d   _DMACH1ModeConfig
00338a97   _StartDMACH1
00338a9f   _DMACH2AddrConfig
00338ab1   _DMACH2BurstConfig
00338ac1   _DMACH2TransferConfig
00338ad1   _DMACH2WrapConfig
00338ae4   _DMACH2ModeConfig
00338b3e   _StartDMACH2
00338b46   _DMACH3AddrConfig
00338b58   _DMACH3BurstConfig
00338b68   _DMACH3TransferConfig
00338b78   _DMACH3WrapConfig
00338b8b   _DMACH3ModeConfig
00338be5   _StartDMACH3
00338bed   _DMACH4AddrConfig
00338bff   _DMACH4BurstConfig
00338c0f   _DMACH4TransferConfig
00338c1f   _DMACH4WrapConfig
00338c32   _DMACH4ModeConfig
00338c8c   _StartDMACH4
00338c94   _DMACH5AddrConfig
00338ca6   _DMACH5BurstConfig
00338cb6   _DMACH5TransferConfig
00338cc6   _DMACH5WrapConfig
00338cd9   _DMACH5ModeConfig
00338d33   _StartDMACH5
00338d3b   _DMACH6AddrConfig
00338d4d   _DMACH6BurstConfig
00338d5d   _DMACH6TransferConfig
00338d6d   _DMACH6WrapConfig
00338d80   _DMACH6ModeConfig
00338dda   _StartDMACH6
00338de2   _INT13_ISR
00338dec   _INT14_ISR
00338df6   _DATALOG_ISR
00338e00   _RTOSINT_ISR
00338e0a   _EMUINT_ISR
00338e14   _NMI_ISR
00338e1e   _ILLEGAL_ISR
00338e28   _USER1_ISR
00338e32   _USER2_ISR
00338e3c   _USER3_ISR
00338e46   _USER4_ISR
00338e50   _USER5_ISR
00338e5a   _USER6_ISR
00338e64   _USER7_ISR
00338e6e   _USER8_ISR
00338e78   _USER9_ISR
00338e82   _USER10_ISR
00338e8c   _USER11_ISR
00338e96   _USER12_ISR
00338ea0   _SEQ1INT_ISR
00338eaa   _SEQ2INT_ISR
00338eb4   _XINT1_ISR
00338ebe   _XINT2_ISR
00338ec8   _ADCINT_ISR
00338ed2   _TINT0_ISR
00338edc   _WAKEINT_ISR
00338ee6   _EPWM1_TZINT_ISR
00338ef0   _EPWM2_TZINT_ISR
00338efa   _EPWM3_TZINT_ISR
00338f04   _EPWM4_TZINT_ISR
00338f0e   _EPWM5_TZINT_ISR
00338f18   _EPWM6_TZINT_ISR
00338f22   _EPWM1_INT_ISR
00338f2c   _EPWM2_INT_ISR
00338f36   _EPWM3_INT_ISR
00338f40   _EPWM4_INT_ISR
00338f4a   _EPWM5_INT_ISR
00338f54   _EPWM6_INT_ISR
00338f5e   _ECAP1_INT_ISR
00338f68   _ECAP2_INT_ISR
00338f72   _ECAP3_INT_ISR
00338f7c   _ECAP4_INT_ISR
00338f86   _ECAP5_INT_ISR
00338f90   _ECAP6_INT_ISR
00338f9a   _EQEP1_INT_ISR
00338fa4   _EQEP2_INT_ISR
00338fae   _SPIRXINTA_ISR
00338fb8   _SPITXINTA_ISR
00338fc2   _MRINTB_ISR
00338fcc   _MXINTB_ISR
00338fd6   _MRINTA_ISR
00338fe0   _MXINTA_ISR
00338fea   _DINTCH1_ISR
00338ff4   _DINTCH2_ISR
00338ffe   _DINTCH3_ISR
00339008   _DINTCH4_ISR
00339012   _DINTCH5_ISR
0033901c   _DINTCH6_ISR
00339026   _I2CINT1A_ISR
00339030   _I2CINT2A_ISR
0033903a   _SCIRXINTC_ISR
00339044   _SCITXINTC_ISR
0033904e   _SCIRXINTA_ISR
00339058   _SCITXINTA_ISR
00339062   _SCIRXINTB_ISR
0033906c   _SCITXINTB_ISR
00339076   _ECAN0INTA_ISR
00339080   _ECAN1INTA_ISR
0033908a   _ECAN0INTB_ISR
00339094   _ECAN1INTB_ISR
0033909e   _XINT3_ISR
003390a8   _XINT4_ISR
003390b2   _XINT5_ISR
003390bc   _XINT6_ISR
003390c6   _XINT7_ISR
003390d0   _LVF_ISR
003390da   _LUF_ISR
003390e4   _PIE_RESERVED
003390ee   _rsvd_ISR
003390f8   _InitEPwm
003390fd   _InitEPwmGpio
00339106   _InitEPwm1Gpio
00339118   _InitEPwm2Gpio
0033912a   _InitEPwm3Gpio
0033913e   _InitEPwm4Gpio
00339152   _InitEPwm5Gpio
00339164   _InitEPwm6Gpio
00339176   _InitEPwmTimer
003393ac   _StartePWMTimers
003393b4   _free
003393f9   _minit
0033941f   _malloc
00339475   _realloc
0033952c   _max_free
0033954e   _free_memory
0033956c   _chkheap
0033956e   _calloc
00339588   _InitMcbsp
0033958d   _InitMcbspa
003395b9   _InitMcbspb
003395e5   _InitMcbspa8bit
003395ec   _InitMcbspa12bit
003395f7   _InitMcbspa16bit
00339602   _InitMcbspa20bit
0033960d   _InitMcbspa24bit
00339618   _InitMcbspa32bit
00339623   _InitMcbspb8bit
0033962a   _InitMcbspb12bit
00339635   _InitMcbspb16bit
00339640   _InitMcbspb20bit
0033964b   _InitMcbspb24bit
00339656   _InitMcbspb32bit
00339661   _InitMcbspGpio
00339666   _InitMcbspaGpio
003396a0   _InitMcbspbGpio
003396c8   _delay_loop
003396de   _clkg_delay_loop
003396f4   _InitECan
003396fb   _InitECana
0033977c   _InitECanb
003397fd   _InitECanGpio
00339802   _InitECanaGpio
00339818   _InitECanbGpio
00339828   _InitXintf
0033987d   _InitXintf32Gpio
003398c4   _InitXintf16Gpio
0033991e   _InitSysCtrl
00339927   _ServiceDog
00339931   _DisableDog
00339939   _InitPll
00339985   _InitPeripheralClocks
003399e0   _CsmUnlock
00339a11   _InitAdc
00339a27   _InitProjectAdc
00339a91   _InitECap
00339aa2   _InitECapGpio
00339aa5   _InitECap1Gpio
00339ab3   _InitECap2Gpio
00339ac2   _InitECap3Gpio
00339ad0   _InitECap4Gpio
00339ade   _InitECap5Gpio
00339aec   _InitECap6Gpio
00339afa   _StarteCAPTimers
00339b09   _InitDSP_IORegs
00339b2d   _InverterPWMOn
00339b42   _InverterPWMOff
00339b50   _DisableUnusedPWMs
00339b5c   _SetIOGood
00339bd1   _WatchdogReset__Fv
00339be6   _FastShutdown__Fv
00339bf1   _InitWatchdog
00339bff   _DisableWatchdog__Fv
00339c0b   _InitEPLDWatchdogEcho
00339c30   _InitEQep
00339c31   _InitEQepGpio
00339c36   _InitEQep1Gpio
00339c60   _InitEQep2Gpio
00339c86   _InitCpuTimers
00339c9c   _ConfigCpuTimer
00339cd7   _InitSci
00339cd8   _InitSciGpio
00339cdf   _InitSciaGpio
00339cf4   _InitScibGpio
00339d08   _InitScicGpio
00339d1e   _c_int00
00339d64   _main
00339d96   _InitPieCtrl
00339db5   _EnableInterrupts
00339dbe   _InitSpi
00339dbf   _InitSpiGpio
00339dc2   _InitSpiaGpio
00339de4   ___memcpy_ff
00339e05   _InitPieVectTable
00339e25   ___nw__FUl
00339e44   __args_main
00339e5d   C$$EXIT
00339e5d   _abort
00339e5f   _exit
00339e76   _InitGpio
00339e8d   _InitI2C
00339e8e   _InitI2CGpio
00339ea4   _MemCopy
00339eb9   __register_unlock
00339ebd   __register_lock
00339ec1   __nop
00339eca   _DSP28x_DisableInt
00339ece   _DSP28x_RestoreInt
00339ed1   ___dl__FPv
00339ed6   _SetDBGIER
00339ed9   ___default_new_handler__Fv
00339eda   ___cinit__
00339eda   ___etext__
00339eda   cinit
00339eda   etext
0033a026   _PieVectTableInit
0033fff6   code_start
00380080   _ADC_cal
ffffffff   ___binit__
ffffffff   ___c_args__
ffffffff   ___pinit__
ffffffff   binit
ffffffff   pinit

[457 symbols]
